:10000000FEC6000018C700000C943A1514C7000083
:1000100012C700000C94C0180EC700000CC70000E7
:100020000AC700000C944C1D06C7000004C700005E
:1000300002C7000000C70000FEC60000FCC60000AA
:10004000FAC60000F8C60000F6C60000F4C60000BC
:10005000F2C600000C94531FEEC60000ECC6000070
:10006000EAC60000E8C60000C00000000000B600BC
:10007000D608D008C600C1084608CF0096072F084A
:10008000D500A3079B08E500AB077508F200B3078E
:100090003E080001BB075A080901C80720081601DD
:1000A000D7074E082601E40711083201F2070208BB
:1000B000000000000000456967656E652049440046
:1000C0005345545550004B6F6E7472617374004CFD
:1000D00069636874005369676E616C3A204D65739B
:1000E00073616765005369676E616C3A205573658B
:1000F000720053656E64657665727375636865003A
:100100004672657175656E7A00435120656D706643
:10011000616E67656E0042616B656E20496E746545
:100120007276616C6C005265706561742D466C610D
:1001300067004645430048415550544D454E5500D3
:100140004D48656172640056657266617373656ED1
:10015000004E6163687269636874656E004572770A
:1001600065697465727400536574757000417573C8
:10017000736368616C74656E0036010000000040B6
:1001800001DB0900004701BD0900005101B9090068
:10019000005D01AC0900006701B20900006D016D4E
:1001A000090000000000000000DD0100000000E781
:1001B000011B0A0000D301FC090000EE01E909005F
:1001C000000002E00900000C02DE0900000000004F
:1001D000000000456D7066E46E676572005645521A
:1001E00046415353454E0053656E64656E00456E3F
:1001F00074777572662073706569636865726E00E6
:1002000054657874206C656572656E004265656E34
:1002100064656E0044657461696C73005D02000082
:10022000000046027E0A000050026E0A00006702CB
:10023000620A00007502670A00001402640A0000E6
:10024000000000000000416E74776F7274656E00EC
:100250005765697465726C656974656E004E4143DB
:100260004852494348540045726E65757420736561
:100270006E64656E004CF6736368656E0053656E60
:1002800064656E009C02000000007D029B0A000075
:10029000A3029D0A00000000000000004D484541F7
:1002A0005244004C69737465206C656572656E001C
:1002B000000108080900213C221F243E21322A2582
:1002C000222A150C083F2E2A131C2A11023A0F1459
:1002D0002A15042A1D290814232214093C0A3D3E2C
:1002E0002A151C22233E221D3E2A233E0A031C22DD
:1002F0003B3E083F223E2310201F3E08373E202170
:100300003E0C3F3E043F1C221D3E0A051C323D3E72
:100310000A352C2A1B023E033E203F1E201F3E189A
:100320003F360837063807322A2732283B000001BB
:10033000BEBF0E000E0128FE2828FE294C9EF29E0C
:10034000F2650C12522C10689490616CFE92BE6C97
:10035000E0990403387CC68382C67C3914083E08C1
:100360001508083E08093071101011C0C1C0300FC7
:100370007CFE8282FE7D84FEFE818CC2E2B29E8D76
:1003800044829292FE6D302824FEFE214E8E8A8A8F
:10039000FA737CFE9292F2610202E2FA1E076CFE90
:1003A0009292FE6D0C9E92D27E3DEC0D6C6D3030C3
:1003B00048488485282828282984844848303104DE
:1003C000A2B21E0D384492BAAA9ABA2419E0F83E95
:1003D000263EF8E1FEFE9292FE6D7CFE8282C645CC
:1003E000FEFE8282FE7DFEFE929283FEFE121203CC
:1003F0007CFE8292F2F5FEFE101010FEFF82FEFEE1
:10040000838082FE7FFEFE386CC683FEFE80808184
:10041000FEFE0E1C38180CFEFFFE0E1C3870FF7C12
:10042000FE828282FE7DFEFE22223E1D3C7E4262D4
:10043000C2FEBDFEFE3272DE8D4C9EBAF265020235
:10044000FEFE02037EFE8080FE7F0E3EF0F03E0F39
:100450003EFEC03E3EC0FE3FC6EE3838EEC7061E2A
:10046000F8F81E07E2F2BA9E8FFEFE82830638C1BC
:100470008282FEFF0804020204098080808080815D
:10048000020540E8A8F8F1FEFE88F87170F8888946
:1004900070F888FEFF70F8A8B8B1FCFE0A0310B827
:1004A000A8F879FEFE08F8F1FAFB88FA7BFEFE70E8
:1004B000D889FEFFF8F808F8F008F8F1F8F808F81D
:1004C000F170F888F871F8F8283811103828F8F920
:1004D000F8F8101990B8E8497CFC8978F880F8F9A8
:1004E0001878E0781938F8C030C0F839D8F820F812
:1004F000D918B8E07819C8E8B899E3F83E263EF86C
:10050000E77AFE848484FE7B7AFA8080FA7B42EA72
:10051000A8FAF372FA88FA737AFA80FAFBFC7E92F0
:10052000FE6D000001BF0E000F20E83E28F82E09E6
:100530008894FEA4454626100864636C92926C5021
:100540008104020138448382443914083E081508A6
:10055000083E0809C1202141C038077C82827D8481
:10056000FE81C2A2928D8292926D302824FE219E3D
:100570009292637C92926182621A076C92926D0CE5
:1005800092927D8069D920505050895050505050DF
:1005900051885050502102A2120D384492AABA2418
:1005A00019E0382638E1FE92926D7C82828245FE07
:1005B00082824439FE929283FE1212037C829292CE
:1005C000F5FE10101010FF82FE8380827FFE10283F
:1005D0004483FE808081FE0618601806FFFE040832
:1005E0001020FF38448282824439FE2222221D38A4
:1005F0004482A242C4B9FE1232528D8C929292630E
:100600000202FE02037E808080807F0E30C0C030F8
:100610000F3EC0380638C03FC6281028C70618E06D
:100620001807C2B28A87FE830638C182FF08040217
:1006300004098080808081020540A8A8F1FE888896
:1006400071708889708888FF70A8A8B1FC12131097
:10065000A8A879FE0808F1FB887BFE205089FFF8E6
:100660000808F00808F1F80808F170888871F8287F
:100670002811102828F9F8100990A8497C89788059
:1006800080F9186080601938C0601860C039D820BF
:10069000D918A0A079C8A899E2382638E33A44824C
:1006A0008282443B7A808080807B40AAA8F3728853
:1006B00088737A8080FBFC02926D2D032205B002C4
:1006C0003003250500003203260500003603290506
:1006D00000003C03300500004203350500004B03D9
:1006E0003B0500005203410500005403440500008F
:1006F0005803470500005C034A05000061034F05ED
:10070000000066035405000068035505B2026B0340
:100710005705B5026D035805000070035B05B7026D
:1007200076035F05BA027A036205BD02800366059F
:10073000C00286036A05C3028C036F05C6029203DA
:100740007305C90298037705CC029E037B05CF028F
:10075000A4037F05D202AC038505D502AA03830555
:100760000000AE038605D602B4038B050000B90372
:100770009105D902BF0396050000C4039A05000045
:10078000CD03A105DC02D403A605DF02DA03AA0526
:10079000E202E003AF05E502E603B405E802EB037D
:1007A000B805EB02F003BC05EE02F603C105F10249
:1007B000FD03C705F4020104CA05F7020504CD05CF
:1007C000FA020B04D205FD021004D6050003190439
:1007D000DD0503031F04E30506032604EA050903F8
:1007E0002C04EF050C033304F6050F033904FB0555
:1007F00012033E04000615034404050618034A04C8
:100800000B061B03500411061E035804180621038F
:100810005E041D06240364042206270369042606D9
:1008200000006D042806000070042B06000074040C
:100830002D0600007A04320600008004370600000E
:1008400082043906DC0287043D06DF028C0441067F
:10085000E20290044406E50295044806E8029A0480
:100860004C06EB029E044F06EE02A3045306F1026F
:10087000A8045706F402AA045806F702AD045A0663
:10088000FA02B2045E06FD02B4045F060003BC0473
:1008900066060303C1046A060603C6046E0609035E
:1008A000CB0472060C03D00476060F03D404790639
:1008B0001203D8047C061503DB047E061803E0044B
:1008C00082061B03E50487061E03EC048E06210343
:1008D000F10491062403F60495062703FA0498060A
:1008E0002A0301059D0600000805A40600000E0568
:1008F000AA062A031305AE0600001805B20600007A
:100900001D05B60600008A0996097E0970092E2C7D
:100910003F2127222D2829402F3A5F3B2B26252ACD
:100920003D3C3E40245B5D5C5E60AAAA2DD4AAAA31
:10093000AA2DD4AA2DD4AA2DD4AA2DD4AAF0CC3372
:100940005A435100554900333537004A756C2032FF
:100950003720323030390032303A35353A323200D1
:10096000204765727269742044483847484800003F
:100970000D102844002844824428004428100B24E9
:100980003E2000322A2400222A140B302838003E50
:100990002810001028280B3C0A3C003E2A14001C9A
:1009A000222207E08890A09088E007E08890AE902F
:1009B00088E007E08884BA8488E007E0868ABE8AF7
:1009C00086E007E080A8A8A880E007E080A890A8BB
:1009D00080E00503053F0503087F4345494945433A
:1009E0007F081C2214001C223C2046694669534D96
:1009F00053657200417573736368616C74656E2032
:100A00003F004E4F43414C4C004E61636872696336
:100A10006874656E0045696E74726167206CF67368
:100A20006368656E3F006D696E004E6F742073657C
:100A300065206D65004D48204C6973746500446500
:100A40007461696C7300416273203A2000456D70D7
:100A5000663A20005A6569743A004B65696E204514
:100A60006D7066E46E6765722067657365747A748D
:100A70002E20416E20616C6C652073656E64656E1E
:100A8000203F00435100416E736568656E006175DB
:100A9000730065696E004D736720696E20506F7337
:100AA000746175732D2067616E672065696E676577
:100AB0007265696874004D657373616765656E740E
:100AC00077757266206162676573706569636865D2
:100AD000727400454E545755524600537065696311
:100AE00068657220766F6C6C21204E696368742093
:100AF000676573706569636865727400416C6C65E5
:100B0000204E6163687269636874656E206CF67369
:100B10006368656E203F004B616C7473746172741E
:100B20002064757263682D2066FC6872656E3F00F4
:100B30004265657000566962726100426565702F9A
:100B4000566962726100204F4B2000204241434BA6
:100B50002000204A612000204E65696E2000203C64
:100B60002D2000205345542000204D454E55452052
:100B700000204D482000204D534720003C2D2000F0
:100B80002D3E20003433342E353030003433392EAE
:100B9000373030003433342E39303000D80B06066D
:100BA000DA0B3703E10B3812E70B390CED0B330B83
:100BB000F20B3211F80B310200000000020C151587
:100BC000040C2A2A060C301B090C23230B0C3613A9
:100BD000110C350A160C341406007071727337DF6D
:100BE0000074757638FC007778797A390064656628
:100BF000330061626332E4002E2C3F2131272D2F18
:100C00003A0015002A0020300023006D6E6F36F682
:100C1000006A6B6C35006768693400554900A90C9F
:100C200000000000B30C2A220000C40C4221000086
:100C3000480CCA210000D10CB5210000500C442101
:100C4000000000000000000056657273696F6E00BE
:100C500048462D5465737466756E6B74696F6E00CB
:100C6000303A204144432D5765727400333A205482
:100C700058206D697420504100323A20525800319A
:100C80003A205458206F686E65205041004154004E
:100C90004259005645520053504549434845524237
:100CA000454C4547554E4720004552574549544508
:100CB000525400537065696368657262656C65675C
:100CC000756E67004C6976652D6D6F6E69746F7215
:100CD000004E6575737461727400000000000000BE
:100CE00000000000000000000000000102030405F5
:100CF000060708090A0B0C0D0E0F00020406080A6D
:100D00000C0E030107050B090F0D000306050C0F60
:100D10000A090B080D0E070401020004080C030762
:100D20000B0F06020E0A05010D0900050A0F070246
:100D30000D080E0B0401090C030600060C0A0B0D2E
:100D400007010503090F0E08020400070E090F082A
:100D500001060D0A030402050C0B0008030B060E26
:100D6000050D0C040F070A02090100090108020B16
:100D7000030A040D050C060F070E000A070D0E04EA
:100D800009030F050802010B060C000B050E0A01F2
:100D90000F04070C02090D060803000C0B070509D8
:100DA0000E020A06010D0F030408000D0904010CD0
:100DB0000805020F0B06030E0A07000E0F010D03B4
:100DC000020C09070608040A0B05000F0D020906AC
:100DD000040B010E0C030807050AFF0001040208BA
:100DE000050A030E0907060D0B0C01020408030691
:100DF0000C0B050A070E0F0D0901F0CC335A112414
:100E00001FBECFEFD8E0DEBFCDBF11E0A0E0B1E064
:100E1000E2EBF9E502C005900D92AA30B107D9F7CF
:100E200015E0AAE0B1E001C01D92A233B107E1F7DD
:100E300019D00C94D72CE4C887E187B980E188B930
:100E400084EF8AB98FEF8BB98EE284B985E085B9DA
:100E500081E58CBD81E08DBD83E08093640080934B
:100E60006D00089514BE88E10FB6F8948093600079
:100E7000109260000FBEE0DF0E94CC1AD7D17894A8
:100E80000E949C180E94AD180E94401F0E94BB1A2D
:100E90000E94E2190E94EB140E94D7190E943F1988
:100EA0008A9741F48CEF9AE060E012D4882311F025
:100EB0000E9422210E940C1D0E94131F0E94F120FB
:100EC0008AB580618ABD0E94DB130E948E1939D3D6
:100ED0008091C9029091CA028038910541F40AB408
:100EE00003FE03C00E94631202C00E94D00F8091D3
:100EF000C9029091CA028050904829F789E791E091
:100F000061E006D5E0CFF999FECF92BD81BDF89A98
:100F100080B50895F999FECF1FBA92BD81BD60BD1D
:100F20000FB6F894FA9AF99A0FBE0895809152017B
:100F300090E080FF91E0809152018E7F892B809319
:100F4000520180E00895809154018F5F83708093F7
:100F5000540180E00895809155018F5F83708093E4
:100F6000550180E00895809156018F5F87708093CE
:100F7000560180E00895809153018F5F8093530163
:100F800080915301833010F01092530180E0089556
:100F90008091520190E082FF91E0990F990F80912A
:100FA00052018B7F892B8093520180E008958091BC
:100FB00057018F5F80935701809157018B3010F05C
:100FC0001092570180E008958091520190E081FFD6
:100FD00091E0990F809152018D7F892B809352016E
:100FE00080E008958091520190E083FF91E0990F95
:100FF000990F990F80915201877F892B809352011D
:1010000080E008959C018091520183FF05C0C901D1
:1010100062E97AE00C94852BC9016EE87AE00C94C1
:10102000852B9C018091520181FF05C0C90162E5B9
:101030007BE00C94852BC90167E57BE00C94852B44
:101040009C018091520182FF05C0C90162E57BE0ED
:101050000C94852BC90167E57BE00C94852B9C01E2
:101060008091520180FF05C0C90162E97AE00C94C9
:10107000852BC9016EE87AE00C94852BBC01809128
:10108000560190E04AE050E00C94202CBC01809185
:10109000510190E04AE050E00C94202CBC0180917A
:1010A000570190E04AE050E00E94202C66E27AE08E
:1010B0000C947A2B9C0180915301882321F4C9015F
:1010C00064E87BE00FC080915301813021F4C901B5
:1010D0006CE87BE007C080915301823029F4C9019C
:1010E00064E97BE00C947A2B08959C018091550172
:1010F000882321F4C9016EE87AE00FC08091550180
:10110000813021F4C90160E37BE007C08091550183
:10111000823029F4C90165E37BE00C947A2B80913D
:101120005501833019F080E090E00895C9016BE328
:101130007BE00C947A2B9C0180915401882321F44C
:10114000C9016EE87AE00FC080915401813021F42A
:10115000C90160E37BE007C080915401823029F42B
:10116000C90165E37BE00C947A2B809154018330B4
:1011700019F080E090E00895C9016BE37BE00C94E6
:101180007A2B809151018E5F8093510180915101A2
:10119000893210F0109251010E94E21980E0089506
:1011A00069E471E048E050E00C94DD2BCF93DF93CD
:1011B000CEE5D1E08FE0FE0111928A95E9F7CE01EC
:1011C00069E471E048E050E00E94DD2BCE0168E068
:1011D00046EB50E020E0CDD4882339F089E491E05B
:1011E000BE0148E050E00E94DD2B80E0DF91CF910E
:1011F000089580915801855980936600F999FECF32
:1012000080E090E069E471E040E150E02AE837E0F6
:101210000E94062C0E943515882331F078940E9494
:1012200035158823E1F7F8940C94EB14CF93DF93F2
:10123000F999FECF89E491E060E070E040E150E090
:1012400023E837E00E94EC2BF999FECFC0E1D0E013
:10125000D2BDC1BDF89A80B58A3209F43BC081E0A5
:10126000809357018BE280935101809152018160FC
:1012700080935201109253018091520182608093B9
:10128000520183E08093560110925401109255014F
:1012900089E491E062E07AE048E050E00E948C2B23
:1012A000F999FECF80E090E069E471E040E150E020
:1012B0002AE837E00E94062CF999FECFF999FECF73
:1012C0001FBAD2BDC1BD8AE280BD0FB6F894FA9AAA
:1012D000F99A0FBEDF91CF9108951F9384EF99E0A3
:1012E00060E0F6D18823A9F11FB7F8948AB58F7E04
:1012F0008ABD8AB58F7D8ABD10928B0010928A00BC
:1013000010928900109288000E94D71984E20E94EE
:10131000CA1980E092E80E947C148BEA80936400F2
:1013200084E00E940B1D1FBF83B7817F866083BF4F
:1013300083B7816083BF889583B78E7F83BF0AB4EC
:1013400004FEF2CF83E8809364000E94E2190E94B9
:10135000EB1481E01F9108958EE19CE061E0D8D20A
:1013600080E0089588E690E060E0D2D242DF80E03D
:1013700008950E94631280E00895EFECF2E08AEA9B
:10138000DF011D928A95E9F78091E102887F8360F1
:101390008093E10290915201929590728F7D892BFA
:1013A0008093E102CF01449666E947E451E021E0F1
:1013B000E0D380E00895F4D581E0089582E00895B7
:1013C00086E9E3EEF2E0DF011D928A95E9F781E01C
:1013D00008958091E102887F81608093E1020E94FC
:1013E000B91C882319F086EB9AE002C08BED9AE0D5
:1013F00061E06ED181E00895CF93DF93CEE5D1E037
:101400008FE0FE0111928A95E9F7CE016FEC72E050
:101410000E94BE2BCE0168E043ED51E020E0A9D34D
:10142000882329F08FEC92E0BE010E94BE2B80E061
:10143000DF91CF910895CF93DF93EFECF2E001902D
:101440000020E9F73197EF5CF240329708F4D4DFDF
:10145000CFECD2E0FE0101900020E9F73197EC1BC0
:10146000FD0B329758F48AE59AE060E031D1882389
:1014700029F1CE0163E87AE00E94852B8091E10298
:10148000887F83608093E1029091520192959072DF
:101490008F7D892B8093E1020E94B91C882319F06B
:1014A00086E99AE002C08BED9AE061E011D188E014
:1014B000EFECF2E0DF011D928A95E9F781E0DF9120
:1014C000CF91089583E008958AD080E0089585E162
:1014D0009AE060E0FDD0811182E00895EFECF2E047
:1014E00088E0DF011D928A95E9F7CF01449666E90D
:1014F00040E552E021E03DD381E008950F931F9332
:101500000FEC12E0C801085F1F4FB80148E050E03F
:101510000E94DD2B045F1F4F86E9F80111928A9526
:10152000E9F7C80166E946E452E021E022D381E010
:101530001F910F91089582E008950E94131F81E08A
:1015400008950AB401FE08C080E060E00E94CE1950
:1015500082ED99E00E94A31A0AB403FE08C087E056
:1015600060E00E94CE1988ED99E00C94A31A0895CA
:101570000F931F93CF93DF938C01EB0180E065E025
:101580000E94CE1982E06EE70E94B619011511057E
:1015900019F0C8010E94581A84E265E00E94CE1931
:1015A0008091CC02E82FF0E0EE0FFF1FEA5FF64FCC
:1015B000859194910E94A31A209761F0CE010E9418
:1015C000811A94E5981B892F65E00E94CE19CE01FF
:1015D0000E94581ADF91CF911F910F910895FF92A9
:1015E0000F931F930E94D719ACDF89E160E00E943E
:1015F000CE1982E060E80E94B61984E192E00E9470
:10160000581A86E49BE06BE47BE0B2DF81E060E0A7
:101610000E94B61980E061E00E94CE1986E49AE04B
:101620000E94581A0EE511E09FE0F92EF8012F2DC7
:1016300011922A95E9F7C80167ED72E048E050E0A1
:101640000E94DD2BC8010E94651A80E062E00E94C2
:10165000CE198DE49AE00E94581AF8012F2D1192AC
:101660002A95E9F7C8016FEC72E048E050E00E946B
:10167000DD2BC8010E94651A80E063E00E94CE194C
:1016800084E59AE00E94581AF8011192FA94E9F759
:101690008091DF029091E002B8014AE050E00E94A0
:1016A000202C0E94651A0E948E198091C902909187
:1016B000CA028050904839F08091C9029091CA02C4
:1016C0008038910581F781E01F910F91FF90089577
:1016D000FF920F931F938C01F62E0E94D71980E082
:1016E00062E00E94CE1980E060E00E94B619C80155
:1016F0000E94581AFF2029F086E49BE060E070E029
:1017000004C082E59BE067E57BE032DF0E948E1932
:101710008091C9029091CA028050904811F481E0F2
:1017200008C08091C9029091CA028038910571F772
:1017300080E01F910F91FF900895EF92FF920F9319
:101740001F93CF93DF93962F682F70E088E2989FC6
:10175000C00111240E94632C22E0E22EE60E00E07C
:10176000FF24C1E0D0E081E56F2D0E94CE1987E013
:101770008E15A8F0002399F48E010E2C02C0000FE4
:10178000111F0A94E2F7802F0E94CC19802F0E942B
:10179000CC19802F8A6A0E94CC1901E00BC080E02E
:1017A0000E94CC1980E00E94CC198AEA0E94CC19D0
:1017B00088EFE80EF39486E0F816A9F6DF91CF9152
:1017C0001F910F91FF90EF900895AF92BF92CF922B
:1017D000DF92EF92FF920F931F93A090CC0283E0D1
:1017E0008093CC0210E0BB2403C01BE101C010E0D9
:1017F0000E94D719A6DE86E49BE06BE47BE0B8DEAE
:10180000EE24DD2428C0EF2DF0E0E25FF64FC49017
:101810001F1531F481E06FEF0E94B619BC2C04C093
:1018200081E060E00E94B619802F6E2D0E94CE19D3
:1018300080E20E943C1A8C2D0E943C1A80E20E9499
:101840003C1AF394055F0D34F1F6E39487E0D80E6B
:1018500084E0E81619F0FD2C00E0D5CF0E948E1927
:101860008091C9029091CA020E94D5188C3009F467
:10187000BCCF8D3088F48630D9F1873038F482308F
:1018800009F4B5CF833009F0B3CF30C08A3081F18D
:101890008B3009F0ADCF10C08331A9F0843130F422
:1018A0008131F1F0823109F0A3CF12C0843131F0DF
:1018B000853109F09DCF1FC016E09ACF112309F49E
:1018C00094CF115095CF1B3108F091CF1F5F90CF6F
:1018D000195F1C3108F48CCF17501830E8F788CF07
:1018E000173010F41B5E84CF175082CF15E180CFE4
:1018F000A092CC0203C0A092CC02BB248B2D1F91DE
:101900000F91FF90EF90DF90CF90BF90AF90089530
:101910002F923F924F925F926F927F928F929F92FF
:10192000AF92BF92CF92DF92EF92FF920F931F93ED
:10193000DF93CF9300D000D00F92CDB7DEB74C012C
:101940006983552436E0252D2F5F239FF001112454
:10195000E80DF91D85919491892B11F0522EF3CF4A
:1019600044244394BB24B394F401859194919B83C4
:101970008A83252C332493E09093CC020E94D719BC
:10198000E0DD89E160E00E94CE1982E060E80E941B
:10199000B6198A819B810E94581AAB2CAA94852D76
:1019A0006A2DCBDEA981AA2309F039C083E69BE02A
:1019B0006BE47BE0DDDD80E060E00E94B61980E052
:1019C00062E00E94CE19B6E0BB9E80011124080D92
:1019D000191DF801859194910E94581AF8013496C6
:1019E000059114910115110509F464C081E060E0CE
:1019F0000E94B61910925E018EE591E0F8010995FA
:101A00008EE591E00E94931AE1E5E81B8E2F63E0DA
:101A10000E94CE198EE591E00E94651A4BC0F981B3
:101A2000F13009F047C086E49BE06BE47BE0A0DD89
:101A30006B2C7724842D90E00396861597051CF473
:101A40005DEF452E4B0CB41408F44B2CC42CDD2454
:101A5000C601880F991F8C0D9D1D880F991F880D39
:101A6000991D9D838C8300E010E07801EC0CFD1C37
:101A70002E143F04FCF0602F6F5F80E00E94CE19AF
:101A8000E614F70419F481E06EEF02C081E060E033
:101A90000E94B619EC81FD81859194910E94581A9B
:101AA0000F5F1F4FAC81BD811696BD83AC830430A0
:101AB0001105D9F60E948E198091C9029091CA022F
:101AC0008050944011F0AB2C04C0E1E0EB1508F01D
:101AD000A52C8091C9029091CA028050904211F0C9
:101AE000BA2C07C0A51418F0BB24B39402C0BA2CBA
:101AF000B3948091C9029091CA028038910511F483
:101B000080E01FC08091C9029091CA02049741F001
:101B10008091C9029091CA028050904809F02BCF61
:101B200086E0B89EF0011124E80DF91D32968591EA
:101B30009491009709F41FCFFC010995882309F4BB
:101B40001ACF0F900F900F900F900F90CF91DF91C1
:101B50001F910F91FF90EF90DF90CF90BF90AF90CB
:101B60009F908F907F906F905F904F903F902F90BD
:101B700008952F923F924F925F926F927F928F9231
:101B80009F92AF92BF92CF92DF92EF92FF920F930C
:101B90001F93DF93CF93CDB7DEB728970FB6F89496
:101BA000DEBF0FBECDBF6C01462E1A01298381E036
:101BB0008093CC02FF2499245524262F30E03B83C8
:101BC0002A83215030403D832C830E94D719B9DCF1
:101BD000F60101900020E9F731978E2E8C18211420
:101BE000310489F082E060E80E94B619C1010E94C8
:101BF000811A86953AE2381B832F60E00E94CE1945
:101C0000C1010E94581A82E060E00E94B61982E485
:101C100060E00E94CE19682C77248A819B81861906
:101C2000970969E571E04AE050E00E94202C0E948B
:101C3000651AFF2019F06EE57BE002C06BE47BE0E3
:101C40008981882319F089E69BE002C086E49BE045
:101C50008FDC81E060E00E94B61990E010E000E0C7
:101C6000EE2411C0EC0DFD1D80819E830E94701A30
:101C7000180F9E81123528F4F91609F4E02E9F5FA3
:101C800002C00F5F10E0E92FF0E06E167F0654F7F8
:101C9000802F6E2D52DDF914A0F410E010C0F60173
:101CA000E90DF11D80810E94701A282F812F90E08C
:101CB000820F911D8235910524F4120F9A94992078
:101CC00071F75F1438F5192DEE240EC01815F9F0D0
:101CD000F601E10FF11D80810E94701A080F023594
:101CE00010F41F5F02C0E39400E01F1578F30FC0EB
:101CF00010E0981451F0F601E90DF11D93948081E4
:101D00000E94701A180F1235A0F39A94EA9493E087
:101D10009E1570F3592CEE24BB24AA24B39480E0C2
:101D20006B2D0E94CE1900E010E01FC05F1441F43B
:101D3000EE2031F48FEF0E94CC19A12EEE24E39413
:101D4000EF81F88580810E94701A282F802F90E003
:101D5000820F911D823591058CF4020FEF81F88579
:101D600080810E943C1A53941F5F9601250D311DFE
:101D700038872F83F90180818823C1F6EE2039F45A
:101D8000581429F48FEF0E94CC19EE24E394F4E068
:101D9000BF1621F60E948E198091C9029091CA0245
:101DA000892B09F412CF8091C9029091CA020E9436
:101DB000D518282F833109F497C0843148F4813134
:101DC000E9F1823108F059C0863009F0A7C01BC084
:101DD000853149F0853108F482C0833219F18A32A5
:101DE00009F09CC08DC0FF2009F4BCC0FA948F2D6F
:101DF00090E0BC016F5F7F4F6C0D7D1D8C0D9D1DB4
:101E00000E94BE2BE2CE2981222309F4ADC089EACB
:101E100091E061E07DDD813009F4C0C0823008F4DA
:101E2000D4CEA2C08091CC028F5F0AB400FE02C063
:101E3000837001C081708093CC02C7CEEF2CEA186A
:101E400009F4C3CE1E2D00E0F601E10FF11D8081E3
:101E50000E94701A080F023510F41150A9F78A2D4C
:101E600090E0AC01410F511D2F2D30E0281B390BA4
:101E7000421753078CF1FE2CA8CE1F2D1A1900E033
:101E80000DC0F601E10FF11D80810E94701A080F4C
:101E9000023518F0F12E00E004C01F5F181588F31A
:101EA000F9CFF81451F0F601EF0DF11DF394808194
:101EB0000E94701A080F0235A0F32A2D30E0210F7E
:101EC000311D2615370514F0F82C7FCE8F2D90E0AC
:101ED000281739070CF079CEF12EFA0C76CEFF20B8
:101EE00009F473CEFA9471CE8F2D90E0EC81FD81D0
:101EF0008E179F070CF069CEF81408F066CE30C03C
:101F00000AB400FC06C08091C802882311F020E0CA
:101F100002C05BDC282F8AB58E7F8ABD203208F490
:101F200054CEF41419F00AB400FE04C08AB58160DE
:101F30008ABDFA940AB400FC0FC0942D07C0F601C4
:101F4000E90FF11D8291319680839150F916B8F313
:101F5000F601E80DF11D1182F601EF0DF11D208350
:101F6000F39433CE80E001C081E028960FB6F89458
:101F7000DEBF0FBECDBFCF91DF911F910F91FF90BC
:101F8000EF90DF90CF90BF90AF909F908F907F9019
:101F90006F905F904F903F902F900895FF2415CE43
:101FA0002F923F924F925F926F927F928F929F9269
:101FB000AF92BF92CF92DF92EF92FF920F931F9357
:101FC000DF93CF9300D000D000D0CDB7DEB783E051
:101FD0008093CC02BB24B394552453942EE5222E37
:101FE00021E0322E96E9492E0E94D719AADA89E11A
:101FF00060E00E94CE1982E060E80E94B61985E395
:102000009AE00E94581AAB2CAA948AE06A2D95DBBC
:1020100089E69BE06BE47BE0ABDA8B2C9924852D81
:1020200090E00396881599051CF48DEF582E5B0CF3
:10203000B51408F45B2C252D30E0C9010197AC01E3
:10204000440F551F480F591F440F551F440F551F6C
:102050004C5D5B4F5E834D8300E010E03A83298343
:102060009C838B83E980FA80E00EF11E5BE0E5162D
:10207000F1040CF08EC0602F6F5F80E00E94CE19DB
:10208000E814F90419F482E06EEF02C082E060E027
:102090000E94B6196B807C80600E711EED81FE81FE
:1020A000608171818281938161157105810591053E
:1020B00009F463C00E94351DDC01CB016CE370E0C4
:1020C0000E94632C6C01643671051CF080E091E085
:1020D0002BC0CB016EE571E04AE050E00E94202C5D
:1020E000F10101900020E9F7E056F14019F480E396
:1020F0000E943C1A8EE591E00E94651A8AE30E94D4
:102100003C1AC6016EE571E04AE050E00E94202CC6
:10211000F10101900020E9F7E056F14019F480E365
:102120000E943C1A8EE591E00E94651A80E20E94AE
:102130003C1AE814F90419F481E06EEF02C081E062
:1021400060E00E94B619F1012FE011922A95E9F79B
:10215000B301660F771F660D771D660F771F660F39
:10216000771F685D7B4F8EE591E048E050E00E946C
:10217000DD2B8EE591E00E94651A0F5F1F4F4D81A8
:102180005E81445F5F4F5E834D830430110509F02B
:1021900069CF0E948E198091C9029091CA02805025
:1021A000944019F481E08B1508F0AB2C8091C902A2
:1021B0009091CA028050904231F4F9E0FA1518F07B
:1021C000BA2CB39401C0BA2C8091C9029091CA0272
:1021D00080389105D1F481E026960FB6F894DEBFE1
:1021E0000FBECDBFCF91DF911F910F91FF90EF9068
:1021F000DF90CF90BF90AF909F908F907F906F9027
:102200005F904F903F902F9008958091C9029091D8
:10221000CA028050904809F0E7CE84E892E061E07D
:1022200077DB823009F0E0CE8B2D90E00197BC0186
:10223000660F771F680F791F660F771F660F771F6E
:10224000685D7B4F8FEC92E048E050E00E94DD2B10
:10225000E3EEF2E0242D11922A95E9F783EE92E065
:1022600066E94DE752E021E084DCBECE3F924F921A
:102270005F926F927F928F929F92AF92BF92CF9216
:10228000DF92EF92FF920F931F93CF93DF93EC01B6
:10229000462E81E08093CC025B8868E0662E712C2C
:1022A0006C0E7D1EA42CBB2455E0AA0CBB1C5A95B9
:1022B000E1F742E1842E912C8A0C9B1CCC243AE25B
:1022C000332E8A89877090E08430910534F482300F
:1022D000910584F4019729F506C086309105A4F094
:1022E0000697F9F407C08EE591E063ED7AE00E946D
:1022F000852B17C08EE591E060E87BE00E94852B7E
:1023000081E691E0BE0109C08EE591E06CE77BE0DB
:102310000E94852B81E691E0B30148E050E00E94E5
:10232000DD2B0E94D7190DD989E69BE06BE47BE099
:102330001FD982E060E80E94B6198EE591E00E9404
:10234000931A8695232D281B822F60E00E94CE19B8
:102350008EE591E00E94651A81E060E00E94B61966
:10236000DC2CEE24E39480E06E2D0E94CE19FF2435
:1023700015C08E010D0D111DF80184890E94701A7F
:10238000282F8F2D90E0820F911D8235910544F406
:10239000F20EF80184890E943C1AD394D51448F3B4
:1023A000F4E0EF16F9F6BAD78091C9029091CA020B
:1023B000892B71F08A898770853051F48AB5877FBF
:1023C0008ABD6A89687F64606A8BC4010E94AC1F01
:1023D0008091C9029091CA0224E08030920709F4EA
:1023E00041C0E4E081309E0728F48038910509F06F
:1023F00068CF57C0F0E280309F0729F080509048A6
:1024000009F05FCF02C010E049C08CE192E061E0CA
:102410007FDA823021F4842D0E948A2042C08330EA
:10242000E9F46A89862F8770863019F08230C9F501
:1024300006C0687F6360C4010E94AC1F42CF0E9447
:102440002C1D998B888B8A89887F83608A8BC50134
:10245000BE0144E150E00E94C61F23C0882309F456
:1024600030CF1FC0CC2009F42CCF10E0FE01EC0DC2
:10247000F11D84890E94701A180F123508F021CFBF
:10248000CA94A1F71ECFFE01EC0DF11D84890E94B4
:10249000701A180F123508F014CFC394C51498F3AE
:1024A00010CFDF91CF911F910F91FF90EF90DF90B0
:1024B000CF90BF90AF909F908F907F906F905F90E4
:1024C0004F903F9008952F923F924F925F926F925C
:1024D0007F928F929F92AF92BF92CF92DF92EF92B4
:1024E000FF920F931F93DF93CF93CDB7DEB72A9759
:1024F0000FB6F894DEBF0FBECDBF33243394DD2476
:10250000D39401C0D62C21E130E07724F999FECF95
:1025100032BD21BDF89A80B5811173942F5F3F4F72
:1025200081E02131380791F7772019F48AB5877F48
:102530008ABD93E09093CC023AD703D889E160E05A
:102540002DD782E060E812D789E09AE0B1D76D2CF0
:102550006A94872D662DF1D886E89AE06BE47BE0DB
:1025600007D8ED2DF0E0FC83EB83832D90E00396FC
:102570008E179F071CF45DEF352E3D0CD31408F425
:102580003D2C222400E010E0232D30E03E832D83FB
:10259000872D90E098878F83ED80FE80E00EF11EFE
:1025A000EF81F885EE15FF050CF4A2C0602F6F5F78
:1025B00080E0F4D630E0CC242FEF0DC0F999FECFA7
:1025C000822F90E08F5E9F4F92BD81BDF89AC0B47C
:1025D000C1103F5F2150832F90E08E159F0574F34B
:1025E0002C2D30E045E0220F331F4A95E1F73A8762
:1025F0002987C9016FEC72E04EE150E00E94F71F9D
:102600008FEC92E063E87AE00E94672B2C018091C6
:10261000E102877090E08330910501F184309105EB
:1026200034F48130910561F0029799F512C085303C
:102630009105F1F085309105B4F0069751F521C070
:1026400032EC832E39E0932E23EEA22E22E0B22E1E
:1026500020C09AEB892E99E0992E17C082EB882E24
:1026600089E0982E12C0B2EA8B2EB9E09B2E04C0EE
:10267000AAEA8A2EA9E09A2EF7EDAF2EF2E0BF2E3D
:1026800008C0EAEC8E2EE9E09E2E7FECA72E72E0C9
:10269000B72EC40158D781E060E068D680E2ECD65E
:1026A0008B819C81E816F90641F481E06EEF5ED6DD
:1026B000E985FA85FA83E9832C2CEEE5F1E02FE039
:1026C00011922A95E9F78EE591E0B50148E050E0D6
:1026D0000E94DD2B452819F481EE99E034D78EE570
:1026E00091E0F3D60F5F1F4F0430110509F054CF6E
:1026F00015D68091C9029091CA028050944019F475
:1027000081E08D1508F06D2C8091C9029091CA026C
:102710008050904219F4671408F463948091C902C0
:102720009091CA0280389105D1F480E02A960FB6C4
:10273000F894DEBF0FBECDBFCF91DF911F910F91F7
:10274000FF90EF90DF90CF90BF90AF909F908F90D1
:102750007F906F905F904F903F902F900895809161
:10276000C9029091CA02049741F08091C9029091E8
:10277000CA028050904809F0C5CE222009F4C2CE8A
:1027800089819A816FEC72E044E150E00E94F71F6A
:102790004091E20250E04B5E5F4F89819A816FEC7D
:1027A00072E00E94F71F23E02093CC028FEC92E0AE
:1027B000622D5CDDA7CE1F93CF93DF93F8D50E94E7
:1027C000A10A81E460E0EAD582E060E0CFD5209103
:1027D0009C0430919D0484E690E0AC01249FC001EC
:1027E000259F900D349F900D112460E770E00E94AA
:1027F0004F2CCB01CEE5D1E0BE014AE050E00E9473
:10280000202CFE0101900020E9F7E156F14031F45F
:1028100080E332D68EE230D6CE0107C080915E01D1
:102820002BD68EE229D6CE0101964FD686E524D648
:1028300083E08093CC020AB403FE05C089E69BE0E6
:1028400066E77BE004C089E69BE061E77BE00E94ED
:10285000B80A88E160E0A2D582E060E087D58AEE20
:1028600099E026D680E060E081D5CEE5D1E01FE09A
:10287000FE01412F11924A95E9F7CE0169E471E01A
:1028800048E050E00E94DD2BCE014DD6982F969562
:102890008AE2891B62E082D5CE0117D6FE01119231
:1028A0001A95E9F780915301882329F4CE0164E851
:1028B0007BE00E947A2B80915301813031F48EE5C8
:1028C00091E06CE87BE00E947A2B8091530182308A
:1028D00031F48EE591E064E97BE00E947A2B8CE193
:1028E00063E05CD582E060E041D58EE591E0EDD516
:1028F000DF91CF911F9108954FB7F8949C015D9897
:102900003EBD0DB407FEFDCF8EB5382F2EBD0DB4E4
:1029100007FEFDCF8EB5282F5D9A4FBFC9010895E0
:10292000906AEACF80E090E0E7CF88EC92E8E4DFBD
:1029300080ED97E00197F1F781E89AECDDDF83E81D
:102940009AECDADFEFDF80E090EBD6DF4098419839
:10295000429A8AB58D7F8ABD10920A01089582E05D
:1029600080930A0180919C0490919D04823E910580
:1029700020F040984298419A03C040984198429A6A
:1029800088E092E8B9DF88E392E8B6DF8AB5826032
:102990008ABD08959B01AC01283185E1380780E0AC
:1029A000480780E0580760F460E678EA80E090E04D
:1029B0000E94762CDA01C90101978068966C0AC0E2
:1029C0006CEF72E485E090E00E94762CDA01C90198
:1029D0000197966C91CF88EE93E028EC30E0F901F6
:1029E0003197F1F70197D9F780EE90EC85DF87ED0D
:1029F00090E882DF8CEA92EC7FDF81E89AEC7CDF62
:102A000080E090EE79DF80E098EC76DF87EF94EC61
:102A100073DF8BDF80E197E20197F1F788E097E0C1
:102A20007FDF80915301813019F488E29FE078DFE5
:102A300080915301823019F487EA97E071DF88EAC8
:102A400094E95ADF60E875E280E090E0A3DF80E47B
:102A500098E952DF6ADF66DF8AB18AB95B9A88E05B
:102A60008093690082E08DBB089580910A018111F5
:102A700081E008951F920F920FB60F9211240F93C9
:102A80001F932F933F934F935F936F937F938F93F6
:102A90009F93AF93BF93EF93FF9344DF97FF2AC0B9
:102AA00080910A01813041F0813018F0823011F5B7
:102AB0001DC081E080930A0181E8ADD780E090EBF2
:102AC0001BDF8C0181E095D7802F27D0882319F058
:102AD0002CDF10920A0180910B01823058F0809116
:102AE0003B01882339F481E096D704C0E0D190E01F
:102AF000986B02DFFF91EF91BF91AF919F918F9102
:102B00007F916F915F914F913F912F911F910F9105
:102B10000F900FBE0F901F901895CF92DF92FF92EB
:102B20000F931F93CF93DF93F82EC0900E01D09098
:102B30000F0180911101C82FD0E080913B01082F37
:102B400010E080910B01823009F460C0833030F4D2
:102B5000882371F0813009F088C13EC0843009F4C7
:102B600013C1843008F4C4C0853009F07EC17BC134
:102B7000FE01E259FE4FF0822196CE0104978B3080
:102B80009105A0F482599E4F0E94272B882371F44F
:102B90008091520183FF06C081E080930B0100E029
:102BA00010E07CC18FEF80930B0178C1C130D1055B
:102BB00019F4CC24CA94DC2CC6016F2D0E944F2B33
:102BC0006C01C431D10509F058C1809181018A5E40
:102BD0008093100183E042C1F801E254FB4FF08280
:102BE0000F5F1F4F0331110509F047C182E0809349
:102BF0000B0110923C0110923D0110923F01109286
:102C00003E01C0E0D0E00FE010E037C1FE01E25924
:102C1000FE4FF0822196C130D10519F4CC24CA941C
:102C2000DC2CC6016F2D0E944F2B6C01C431D105E5
:102C300031F483E080930B018CEA80931001CE0184
:102C400083709070892B09F018C1789480913C01B1
:102C500060913D0190E070E062547B4F82599E4F3D
:102C600040E028E00E940F2A282F843030F08FEFB8
:102C700080930B0188EC90E02BC080913C018C5F2D
:102C800080933C0180913D018D5F80933D01809157
:102C90003E0190913F01820F911D90933F018093DF
:102CA0003E01C431D10508F4E8C080918101882338
:102CB000A1F0809181018A5E809310018091810151
:102CC000873908F4DAC08FEF80930B0180EF90E032
:102CD00090933F0180933E01CEC08FEF80930B0114
:102CE00087E990E090933F0180933E01A9D1C5C050
:102CF000FE01E259FE4FF0822196C6016F2D0E941F
:102D00004F2B6C0120911001822F90E0C817D9073A
:102D100009F0B3C0273120F0FE01E459FE4F1082C4
:102D20000115110591F486E990E090933F0180939D
:102D30003E01C114D10429F485E080930B017894FD
:102D40007FD18FEF80930B0196C084E080930B01BD
:102D50008091810190E0880F991F69E070E00E94E6
:102D6000632C6F5F7F4F8B01000F111F060F171F22
:102D700026512093100110923D0110923C011092B7
:102D80004001C0E0D0E079C080913D01E82FF0E043
:102D9000E254FB4FF0828F5F80933D012196C33058
:102DA000D10509F04DC080913D0190E08017910759
:102DB00011F029E009C080913C01909140012091DF
:102DC0001001281B220F291B789480913C016091EF
:102DD0003D014091400190E070E065547B4F8E577B
:102DE0009E4F0E940F2A282F843060F08FEF80932F
:102DF0000B0189EC90E090933F0180933E01C0E08D
:102E0000D0E039C080913C018C5F80933C0190916F
:102E10003C0180914001890F80933C0180913E01EB
:102E200090913F01820F911D90933F0180933E014D
:102E30008091400191E0892780934001C0E0D0E07B
:102E400080913D0190E080179107BCF080EA90E00E
:102E500090933F0180933E01F3D08FEF80930B015D
:102E600000E010E00AC0000008C010920B01C0E0B2
:102E7000D0E000E010E081E001C080E0D0920F01DE
:102E8000C0920E0100933B01C0931101DF91CF91DD
:102E90001F910F91FF90DF90CF900895C0E0D0E098
:102EA0008BCE43DD85E080936D0181E0B4C59091C8
:102EB0002D0280910C01833009F455C0843030F428
:102EC000813089F1823008F03CC00AC0853009F4B5
:102ED0006AC0853008F451C0863009F090C079C0CE
:102EE00080915201E0910D0183FF11C0E33148F45C
:102EF000EF5FE0930D01E150F0E0E25DF64F849169
:102F0000089510920D0181E080930C010CC082E0C5
:102F100080930C01EF5FE0930D01E150F0E0E65D7E
:102F2000F64F8491089520910D012F3028F4E22F5F
:102F3000F0E0E254FB4F2DC010920D0182E080932F
:102F40000C01E0910D01E43048F4EF5FE0930D01D6
:102F5000E150F0E0E65DF64F8491089510920D0186
:102F600083E080930C0120910D01243118F4E22FAD
:102F7000F0E00DC084E080930C0120910D01E22F60
:102F8000F0E0892F90E04496E817F90738F4E65E00
:102F9000FD4F80812F5F20930D01089585E0809380
:102FA0000C0110920D0190910D01923028F4E92F3F
:102FB000F0E0EC53FD4F17C010920D0180915201CB
:102FC00083FD04C087E080930C0117C086E08093E6
:102FD0000C0190910D0180913B01981748F4E92F65
:102FE000F0E0E353FB4F80819F5F90930D010895C4
:102FF00087E080930C0110923B018AEA08951092B9
:103000000D0110920C014DDF8AB58D7F8ABD80E0E5
:1030100008952BDD882329F0789427DD8823E9F7AC
:10302000F89410920C019BCC20DD882319F081E0EC
:1030300090E0089577DC892F99278170907008952A
:10304000CF93DF938EE691E064E479E00E94672BF2
:10305000EC018091520182FD02C020E00AC08EE6A0
:1030600091E061E479E00E94672B20E0892B09F46C
:1030700021E0CD2B51F0222341F48EE691E069E46A
:1030800071E00E94AB2B892B81F44091810150E0CB
:103090004B5E5F4F89E793E06EE671E00E949B2BE9
:1030A0008AB580688ABD81E000C0DF91CF91089524
:1030B000EF92FF920F931F93CF93DF937C0180E0F9
:1030C00098D40FEF1FEFC0E0D0E009C0FE01E65E2C
:1030D000FD4FC80160810E944F2B8C012196F701A2
:1030E000838990E04496C817D90780F380915201F4
:1030F00083FF05C0C7016EEB74E00E948A25109320
:10310000C5020093C40285DF8091520183FF0AC08B
:10311000C70144966DEC74E0F70143890E94F222E6
:1031200080933B0180E077D480E0DF91CF911F91C5
:103130000F91FF90EF90089582E08093CC0210925F
:10314000CA021092C9021092C7021092C602E8E6A3
:10315000F0E080818460808308959FB7F894E8E66A
:10316000F0E0808184608083509A519A58985998F1
:10317000589A599A50988AB18C7F8AB99FBF0895FE
:103180001F920F920FB60F9211248F93EF93FF931C
:10319000E8E6F0E080818B7F8083FF91EF918F9153
:1031A0000F900FBE0F901F9018959C018AB58E7FCF
:1031B0008ABD4FB7F8948FE18093C8028091C60210
:1031C0009091C7028217930749F48091CB028F5FD9
:1031D0008093CB028AB581608ABD02C01092CB0277
:1031E0003093C7022093C6024FBFEFE0E15021F0B9
:1031F0003695279520FFFACF8091CC02833059F481
:103200001092CB02F0E0EE0FFF1FEE0FFF1FE15612
:10321000F44F84910895F0E0823051F41092CB0283
:10322000EE0FFF1FEE0FFF1FE256F44F849108953B
:103230009FB7F894EE0FFF1FEE0FFF1FE456F44FF9
:10324000259134912115310519F49FBF80E008952F
:103250008091CB02F901E80FF11DE491EE2331F4E6
:1032600080E0F8CF8E2F90E00C94982C8093CB02C6
:103270009FBF8091CC028130A9F38E2F08951F93B8
:1032800019B11370133019F480E090E03DC084E070
:10329000B0D38091520180FF06C00AB404FE03C07F
:1032A0008AB580628ABD20E030E0412F10FF0CC05B
:1032B0005C985098519A00005C9A1EBC0DB407FEB1
:1032C000FDCF51988EB5282F41FF0CC05C98509AC5
:1032D000519800005C9A1EBC0DB407FEFDCF5098BB
:1032E0008EB5382F1092680083E08BBB3093480175
:1032F0002093470184E08FD380914701909148014A
:1033000010924801109247011F910895B8DF00976D
:1033100021F09093CA028093C9020895CF93DF935E
:10332000C0E2DEE410C00BB400FE0AC01092CA0274
:103330001092C9028BB58E7FEAE4F0E0818313C05E
:10334000CE010197F1F79BDF892B69F307C00BB41E
:1033500000FC09C0CE010197F1F702C0C0E2DEE433
:10336000D5DF892BA1F7DF91CF91089580931201CA
:103370006093130108952FB7F8949FEE9BB98EBD0B
:103380005A9861115A9A0DB407FEFDCF8EB55C9A1A
:103390002FBF089560E0EFCF61E0EDCF1F93162FB0
:1033A0008058F8DF812F805CF5DF1F910895CF935F
:1033B000DF93C8EFD1E080E0EFDF2197E1F7DF9105
:1033C000CF9108951092130181E0809312014498E7
:1033D00080ED97E0FC013197F1F7449A0197F1F7FE
:1033E00080E29EE40197F1F781E2D4DF8091510100
:1033F000885D8068CFDF86E0CDDF83E1CBDF80E2D0
:10340000C9DF8CE0C7DFD3CF982F8B3718F18F3D02
:10341000D1F0803E38F4863D69F18C3D61F0843C0A
:10342000A1F407C0863F59F08C3F59F0843E69F4FF
:1034300004C09BE70FC09DE70DC09EE70BC09FE750
:1034400009C090E807C091E805C0923818F080E004
:1034500090E00895905283E0989FF00111248091AC
:103460001201E80FF11DEE0FFF1FE654F94F859191
:10347000949108959CE7EECF0F931F93CF93DF9322
:10348000C3DFEC01009761F08E012196F8010491F1
:10349000802F8E7F9091130189277EDF00FFF4CF6C
:1034A0008091130179DFDF91CF911F910F910895E2
:1034B000CF93DF93EC0101C0DFDFFE012196849101
:1034C0008823D1F7DF91CF910895CF93DF93EC015B
:1034D00001C0D2DF89918823E1F7DF91CF91089570
:1034E00093DF009711F440E009C09C01F9012F5FC0
:1034F0003F4FE491422F481BE0FFF8CF842F8F5FAE
:1035000008951F93CF93DF93EC0110E002C0E8DF32
:10351000180FFE01219684918823C9F7812FDF912E
:10352000CF911F9108951F93CF93DF93EC0110E08B
:1035300002C0D6DF180F89918823D9F7812FDF9138
:10354000CF911F910895FF920F931F93CF93DF9315
:10355000EC018C01FC01F49004C02196FE018491E1
:103560001BDF9E01201B2F15C0F3DF91CF911F9110
:103570000F91FF9008951092CD0282EA809380000F
:1035800082E080938100109289001092880010924E
:103590008B0010928A00089510921C0110921E0157
:1035A0001092230410921D010895FF920F931F9310
:1035B000CF93DF938BB58D7F8BBD90E8F92E01E023
:1035C000F999FECFF999FECF802F90E08F5E9F4F43
:1035D00092BD81BDF89A80B5882319F1C82FD0E03B
:1035E00085E0CC0FDD1F8A95E1F7CE016FE171E038
:1035F00044E150E0FCD410913101812F8770863076
:1036000081F48FE191E064E171E048E050E00E94D4
:10361000C52B892B31F4187F1360CE014296612FA0
:103620009BD4FA940E5FFF2059F6DF91CF911F9142
:103630000F91FF9008950F931F93CF93DF930AB4D8
:1036400007FEE8C080918B038695869586958370EA
:1036500090E08130910509F444C083309105B1F0C8
:10366000892B09F0C4C081E893E053D30BB401FC6B
:103670000BC084E191E061E873E048E050E00E9413
:10368000DD2B8BB582608BBD90DFB1C020912A020B
:1036900030912B028091890390918A032817390772
:1036A00009F0A5C08AE192E061E873E048E050E0EB
:1036B0000E94C52B892B09F09AC000911C0110E0D3
:1036C00045E0000F111F4A95E1F70E5E1F4FC8013C
:1036D00024D4682F687F6260C8013ED4109223040E
:1036E00086C001E110E0F999FECF12BD01BDF89A44
:1036F00080B5882329F1C82FD0E035E0CC0FDD1F3D
:103700003A95E1F7CE01429608D48C5F87708230FB
:10371000B8F4CE016FE171E044E150E068D420914B
:10372000890330918A0380912F01909130012817ED
:10373000390731F490918C0380913201981769F127
:103740000F5F1F4F81E00131180769F654C0802FC9
:1037500090E0412F50E025E0880F991F2A95E1F76E
:1037600069E773E013D4802F612F0ED58AB580628C
:103770008ABD8AB588608ABD8BB581608BBD80911A
:10378000540180FF03C080E28093CD0280915401F8
:1037900081FF03C088E08093CE0289E793E063E86D
:1037A0007AE00E94672B892B11F182E292E069E4B2
:1037B00071E048E050E00E94DD2B8AE192E061E890
:1037C00073E048E050E00E94DD2B10922D028091C2
:1037D0002C02886180932C028091890390918A0346
:1037E00090932B0280932A0282E0809323048AB56F
:1037F0008F778ABD0FC080918B03887F856080930F
:103800008B0310918C031B5E812F58D4082F8823C3
:1038100071F39DCFDF91CF911F910F9108950F9379
:103820001F93CF93DF9321D9882309F09DC0809106
:103830002304813009F46CC0813038F0823009F4FF
:1038400089C0833009F090C03BC01FEFF999FECFCB
:1038500080911E018F5F80931E01F999FECF90E049
:103860008F5E9F4F92BD81BDF89A00B5002319F17C
:10387000C02FD0E075E0CC0FDD1F7A95E1F7CE01C7
:1038800042964BD387708330B1F4CE016AE172E087
:103890004AEA50E0ACD300931C018091560190E0BD
:1038A00063E0880F991F6A95E1F780931D0181E01D
:1038B0008093230459C0112309F456C01150C6CF78
:1038C000109223048AE192E060E070E04AEA50E05E
:1038D0000E94A42B82E292E069E471E048E050E0AB
:1038E0000E94DD2B8AE192E06BE17CE048E050E051
:1038F0000E948C2B80912C02877E80932C028091D9
:103900002C02887F836080932C0210922D0229C0A4
:1039100080911D01882351F0815080931D018F5F9C
:1039200090E087709070892BF9F41BC000911C0106
:1039300010E055E0000F111F5A95E1F70E5E1F4F82
:10394000C801EBD2682F687F6660C80105D310926A
:1039500023040AC080911E01815080931E011092A1
:1039600023048AE192E0A4DBDF91CF911F910F91B4
:103970000895FF920F931F938091E102877E8860E4
:103980008093E10287ED92E069E471E048E050E065
:103990000E94DD2BE3EEF2E001900020E9F7E45E07
:1039A000F240E093E20258D09093E0028093DF026D
:1039B0000091E2020B5EFFB6F894802F7FD3182FA0
:1039C000882319F4FFBE80E010C090E0402F50E043
:1039D000E5E0880F991FEA95E1F76FEC72E0D6D227
:1039E000812F602FD1D3FFBE81E01F910F91FF90F7
:1039F000089590913401982B909334019FB7F894D7
:103A0000E1E6F0E080E88083108287E08093B100F7
:103A10001DBC9FBF089508958EE18093370123E078
:103A2000209336018091570190E090933A01809362
:103A3000390116BC10926E0025BD109285001092BF
:103A40008400109238018FE1809335011092B2000A
:103A500081E080937000089580914301909144012A
:103A6000A0914501B0914601089520914301309104
:103A700044014091450150914601261B370B480BEC
:103A8000590BCA01B9012CE330E040E050E00E943C
:103A9000762CCA01B90108951F920F920FB60F92AA
:103AA00011242F933F934F935F936F937F938F9343
:103AB0009F93AF93BF93EF93FF9382E09ADF809140
:103AC000C802882329F41092C7021092C60205C0CA
:103AD0008091C80281508093C8020AB404FE78C065
:103AE0004091350140FF20C02091CD022223E1F01A
:103AF00084E59CE6A4E1BDEA022E04C0B695A79534
:103B0000979587950A94D2F780FF07C088ED90E0DB
:103B1000909389008093880004C0109289001092CD
:103B2000880021502093CD020AB405FE17C0809171
:103B30008A0090918B00809621E0803E920738F4B5
:103B400090938B0080938A00109238011CC08FEFF5
:103B500091E090938B0080938A0015C020918A0099
:103B600030918B0080918A0090918B00409738F0C3
:103B70002051304030938B0020938A0004C0109273
:103B80008B0010928A000AB401FC18C04F3011F06B
:103B90004423A1F42091CE02222381F088EA90E010
:103BA000022E02C0959587950A94E2F780FF02C025
:103BB000409A01C0409821502093CE028091380154
:103BC000815080933801882319F48AB58F7D8ABD8E
:103BD00080913301882309F08BC080913B018823B9
:103BE00009F086C081E080933301789424DD8091D0
:103BF00035018F3009F413DE30913501343101F590
:103C000080915701882309F46EC080913901909109
:103C10003A01009779F480912304882309F063C066
:103C200083E080932304809157012CE3829FC0019D
:103C3000112401C0019790933A018093390153C038
:103C4000332309F050C08091430190914401A09129
:103C50004501B09146010196A11DB11D809343011C
:103C600090934401A0934501B09346018FE1809366
:103C700035010AB404FC1AC0499905C08091680056
:103C8000846080936800FBDA8038910521F480918C
:103C90003601815001C083E0809336018091360166
:103CA000882321F58AB580618ABD20C0E8DA803496
:103CB000910521F480913601815001C083E0809309
:103CC000360180913601882309F400008091370184
:103CD000882329F48EE180933701D2D007C0815028
:103CE0008093370103C03150309335011092330176
:103CF000FF91EF91BF91AF919F918F917F916F91C4
:103D00005F914F913F912F910F900FBE0F901F9099
:103D10001895CF92DF92FF920F931F93CF93DF936B
:103D20006C0100E010E0F02EE801CC0FDD1FC00FA9
:103D3000D11FCC0FDD1FCC0FDD1FBE01685D7B4F97
:103D4000C60148E050E00E94C52B892B59F4FE01C2
:103D5000EC5DFB4F20813181428153818AE008175D
:103D600041F41AC00F5F1F4F0A301105E1F62AE037
:103D700014C08091430190914401A0914501B091FC
:103D80004601821B930BA40BB50B89559240A040B2
:103D9000B04010F4202F25C02F2D8AB580628ABD37
:103DA0008091550180FF03C084E08093CD02809113
:103DB000550181FF16C086E08093CE0212C02A30E2
:103DC00070F4239FC0011124DC01AC5DBB4FFC01EA
:103DD000E85EFB4F8CE001900D928150E1F721509D
:103DE00001C03CE0222359F788E294E0B60148E0A4
:103DF00050E00E94DD2B8091430190914401A091FD
:103E00004501B09146018093240490932504A0932A
:103E10002604B0932704DF91CF911F910F91FF905B
:103E2000DF90CF9008950F931F93CF93DF93E4E239
:103E3000F4E088E7DF011D928A95E9F78F01C0E081
:103E4000D0E0F8011082118212821382CE01880F15
:103E5000991F8C0F9D1F880F991F880F991F885DD0
:103E60009B4F62E07AE00E94852B2196045F1F4FF2
:103E7000CA30D10531F7DF91CF911F910F9108958D
:103E800080E880BF3D9AE4E6F0E080818E7F808309
:103E900010929D0410929C0487E480937C008DED29
:103EA00080937A0008951F920F920FB60F921124FB
:103EB0008F939F933D988091780090917900813500
:103EC000910540F0809178009091790090939D0445
:103ED00080939C0480917A008F7780937A00809100
:103EE00064008160809364009F918F910F900FBE5A
:103EF0000F901F9018958EBD0DB407FEFDCF08954D
:103F00005F9885E0F8DF80E0F6DF5F9A0EB400FC92
:103F1000F7CF82E08A95F1F70895FF920F931F93F0
:103F20008C01FFB6F894ECDF5F9883E0E4DF812F2B
:103F3000E2DF802FE0DF80E0DEDF5F9AFFBE8EB53C
:103F40001F910F91FF9008955F9886E0D4DF5F9AEC
:103F500082E08A95F1F70895EF92FF920F931F93F5
:103F60008C01F62EEFB6F894CBDFEEDF5F9882E09F
:103F7000C2DF812FC0DF802FBEDF8F2DBCDF5F9AB5
:103F8000EFBE1F910F91FF90EF900895DF92EF9297
:103F9000FF920F931F93CF93DF93EC017B018A0174
:103FA000DFB6F894ADDFD0DF5F9882E0A4DF8D2F1D
:103FB000A2DF8C2FA0DFF70181917F019CDF0150F0
:103FC00010402196CE018F719070892B19F0011548
:103FD000110589F75F9A0115110521F7DFBEDF9101
:103FE000CF911F910F91FF90EF90DF900895DF9296
:103FF000EF92FF920F931F93CF93DF938C017B017E
:10400000EA01DFB6F8947CDF5F9883E074DF812FEC
:1040100072DF802F70DF07C080E06DDF8EB5F701A3
:1040200081937F0121972097B9F75F9ADFBEC7017F
:10403000DF91CF911F910F91FF90EF90DF90089546
:10404000CF93DF93282F342F662311F480E033C001
:10405000862F90E0019760E270E00E94632C6F5F12
:1040600041E050E026C0922F9770822F869586956A
:104070008695A82FB0E0FD01E256FB4FE081892F25
:10408000332349F0EA0102C0CC0FDD1F8A95E2F725
:10409000CE018E2B09C0EA0102C0CC0FDD1F8A952C
:1040A000E2F7CE0180958E23A256BB4F8C932F5FF3
:1040B00061506623C1F6DF91CF91089590E001979A
:1040C00060E270E00E94632C6F5F40E031E0E32F1C
:1040D000E695E695E695F0E0E256FB4F808190E0AC
:1040E000232F277002C0959587952A95E2F780FDCA
:1040F00007C04F5F461729F4832F841B8F5F0895F5
:1041000040E03F3F11F03F5FE2CF8AB580648ABD57
:1041100080E008950F931F93182F21E130E0F99963
:10412000FECFF999FECF32BD21BDF89A80B5811737
:1041300001F50FB7F894F999FECFF999FECF1FBAA0
:1041400032BD21BD10BC0FB6F894FA9AF99A0FBE91
:10415000812F90E025E0880F991F2A95E1F743967B
:10416000DCDE682F6C5E812F40E06ADF0FBF81E0EC
:1041700008C081E02031380719F02F5F3F4FCFCFC3
:1041800080E01F910F910895782F20E031E001C069
:104190009A01F999FECFA90141505040CA018F5EA2
:1041A0009F4F92BD81BDF89A80B5882389F381E045
:1041B0002030380711F480E00895F999FECFF9997D
:1041C000FECF1FBA2F5E3F4F32BD21BD70BD0FB66F
:1041D000F894FA9AF99A0FBE872F41E031DF81E017
:1041E00008951F93CF93DF9380E2EEE9F4E0DF01BF
:1041F0001D928A95E9F781E080939E04C1E1D0E0A9
:10420000F999FECFF999FECFD2BDC1BDF89A10B58C
:10421000112379F0812F90E035E0880F991F3A95AE
:10422000E1F743967ADE682F6C5E19F0812F41E04A
:1042300007DF2196B1E0C131DB0711F7DF91CF91A4
:104240001F9108951F931FB7F89420E030E0822F4C
:10425000F999FECFF999FECF1FBA90E08F5E9F4F7C
:1042600092BD81BD10BC0FB6F894FA9AF99A0FBEB0
:104270002F5F3F4F81E02030380749F7B2DF1FBF83
:104280001F91089580E0089592D882E060E86ED88A
:104290008FE060E083D880E59CE00AD90E94A10A03
:1042A00081E060E063D880E061E078D88FE79CE04F
:1042B000FFD880E062E072D889E79CE0F9D880E01E
:1042C00063E06CD88CE69CE0F3D880E064E066D8CC
:1042D00080E69CE0EDD886E49BE060E070E00E9420
:1042E000B80A1CD88091C9029091CA0280509240AD
:1042F00019F4E9980E94AF148091C9029091CA0202
:104300008050944031F40E9495140E94921482E0EF
:104310008DBB8091C9029091CA028050984029F4C7
:10432000E9980E94AF144198429A8091C9029091F5
:10433000CA02809781F481E464E030D880919C04C3
:1043400090919D046EE571E04AE050E00E94202CBF
:10435000BCD80E948E198091C9029091CA028050E7
:10436000904809F091CF80E0089587E19BE060E0FC
:104370000E94680B882369F0F89428E088E190E0B7
:104380000FB6F894A895809360000FBE209360004C
:10439000FFCF08950CD882E060E80E94B61984E14E
:1043A00060E00E94CE1988E49CE082D880E061E061
:1043B0000E94CE1983E99CE07BD881E060E00E94F6
:1043C000B61980E259D88AEE99E072D880E254D8C2
:1043D00087E499E06DD880E062E00E94CE1982E027
:1043E00060E80E94B61980E99CE062D881E060E054
:1043F0000E94B61980E240D880E699E059D882E060
:1044000060E80E94B61980E063E00E94CE198DE852
:104410009CE04ED882E060E00E94B61980E22CD881
:104420008BE499E045D880E227D887E599E040D829
:1044300086E49BE060E070E00E94B80A0E948E195A
:104440008091C9029091CA028050904809F0A2CF91
:1044500080E00895EF92FF920F931F93CF93DF9325
:104460000E94D71985E060E00E94CE1982E060E8E2
:104470000E94B61987E99CE01BD883E061E00E94A6
:10448000CE1901E0C0E0D0E081E0E82EF12CCE01B1
:104490006FE370E00E944F2C892BD9F4209749F0EC
:1044A00080E00E94CC198FEF0E94CC198FEF0E9400
:1044B000CC19102F1F5F83E0602F0E94CE198FEF61
:1044C0000E94CC198FEF0E94CC1980E00E94CC1979
:1044D000012FCE0168E070E00E94632CDC01CB016B
:1044E000970102C0220F331FAA95E2F782569B4F15
:1044F000FC01808190E0822393238217930711F4BB
:104500008CE901C080E80E94CC192196F1E0C0300E
:10451000DF0709F0BCCF80E00E94CC198FEF0E942A
:10452000CC198FEF0E94CC1982E06EE70E94B61979
:1045300080E065E00E94CE1986E49BE00E94581A54
:104540000E948E1980E0DF91CF911F910F91FF9013
:10455000EF9008958295807F682BEAEDFCE0E60FEE
:10456000F11DE4918E2F08958295807F682B8AED4E
:104570009CE0FC01E60FF11DE4914295407FE42BA5
:104580008E0F911DFC0184910895EAEDFDE0E80F86
:10459000F11DE4918E2F0895EAEEFDE0E80FF11D84
:1045A000E4918E2F08951F93182F613071F0862F9C
:1045B000ECDF9FE0981B892FEFDF1295107F182BFF
:1045C000E12FF0E0E652F34F84911F910895982F68
:1045D0009295907F982BEAEDFCE0E90FF11DE491B4
:1045E0008E2F08952F923F924F925F926F927F92FB
:1045F0008F929F92AF92BF92CF92DF92EF92FF92F3
:104600000F931F93DF93CF93CDB7DEB728970FB6E5
:10461000F894DEBF0FBECDBF3C017B836A83842E3E
:104620001B01198225C1D3011D91B887AF83B981C0
:10463000BB2349F4EFE0DE2ED122E12EE2947FE0AD
:10464000E722EBEF0AC0D12ED2946FE0D622D3013D
:104650001196EC90BFE0EB22ECEF8E0E8FE06D2D0B
:1046600079DFF82E87E06E2D75DF182F6E2D6D2502
:1046700089E070DFA82EA29450EFA5221F25A12A61
:1046800085E06D2D67DFC82E83E06E2D63DF182F68
:1046900088E06D2D5FDF082F8CE06E2D5BDF082733
:1046A0000295007F1C25012B8AE06E2D53DF182F09
:1046B0008D2D67E04FDFE8268CE06E2D4BDF982EC6
:1046C000929440EF94221F25912A4F805884089499
:1046D000411C511CBB24B394AF81B8858C91B98126
:1046E000BB2339F4282F2F70982F92959F70320199
:1046F00007C0282F22952F703201F20190819F7000
:104700003FE0F32EFA20F22687E06F2D9E8322DF12
:104710001A2D12951F7018279E811927812F67E087
:1047200019DFE82E8F2D69E015DFD82E812F69E083
:1047300011DFA82E8F2D63E00DDF902F907FA8262C
:10474000A29480EFA822A9260F70DE240D25A02AAE
:104750008F2D6CE0FFDEE82E812F63E0FBDEC82E9C
:10476000812F6CE0F7DED82E8F2D6AE0F3DE992DD5
:10477000907F082F0D250295007F0927FFE09F22DB
:10478000CE249C240929812F6AE0E4DE9D2C92949A
:1047900010EF9122E8269E28B3940894411C511CE6
:1047A0004F8158854F5F5F4F58874F8354E0B51650
:1047B00009F092CFD3011C91B981BB2319F4612F69
:1047C0006F7006C0612F62956F700894611C711C38
:1047D000E981F1E0EF27E9831A2D1F701627812F59
:1047E00067E0B8DEB82E812F69E0B4DEE82E812FB5
:1047F0006CE0B0DEC82E812F63E0ACDE582EDD24E5
:10480000812F6AE0A7DE202F30E02F703070FF2468
:104810002E253F25B4E0220F331FBA95E1F7A2946D
:10482000AFE0AA22AB24A22AD101AC92292D30E01C
:104830002F7030702C253D25F4E0220F331FFA95A0
:10484000E1F702950F700525022B11960C93119735
:104850009294EFE09E22982674E0CC0CDD1C7A95B1
:10486000E1F79C2812969C92E3E0F0E02E0E3F1EAA
:10487000522CFA815F1A24E0281508F4D4CE882D32
:1048800090E04981840F911D892B09F429C188206A
:10489000E1F0D3011D91B887AF83482D4150B98114
:1048A000BB2341F46FE0D62ED122E12EE2945FE0EB
:1048B000E52209C0D12ED2943FE0D322D301119634
:1048C000EC90BFE0EB22B42E0BC0F301D190F8873F
:1048D000EF83D2942FE0D222BB24BA94EE24198223
:1048E0008FE06D2D37DEF82E87E06E2D33DE182F2A
:1048F0006E2D6D2589E02EDE982E929490EF9922F0
:104900001F25912A85E06D2D25DEC82E83E06E2DB2
:1049100021DE182F88E06D2D1DDEA82E8CE06E2D77
:1049200019DEA826A29480EFA8221C25A12A8AE0DD
:104930006E2D10DE182F8D2D67E00CDEE8268CE042
:104940006E2D08DE882E829400EF80221F25812A9A
:1049500077247394BB20C9F0EF81F88521914B2D0A
:1049600041505981552341F4322F3F70022F029557
:104970000F70F887EF8307C0322F32953F70F887AA
:10498000EF8300810F70B42E0FC08981882319F442
:1049900030E000E009C0AF81B8853D91B887AF83B2
:1049A00032953F7000E01982BFE0FB2EF920F3261C
:1049B00087E06F2DCFDD192D12951F701827102756
:1049C000812F67E0C7DDE82E8F2D69E0C3DDD82E8B
:1049D000812F69E0BFDD982E8F2D63E0BBDD9A2D1E
:1049E000907F98269294A0EF9A229926BFE0AB225E
:1049F000DE24AD249A288F2D6CE0ACDDE82E812FCB
:104A000063E0A8DDC82E812F6CE0A4DDD82E8F2DA9
:104A10006AE0A0DD982D907FA82EAD24A294F0EF3F
:104A2000AF22A926EFE08E22CE248C24A828812F45
:104A30006AE090DD8D2C8294E0EF8E22E8268E28AD
:104A40007394F4E07F1609F085CF7FE0D72ED9204C
:104A50008D2D67E07FDDB82E8D2D69E07BDD182F71
:104A60008D2D6CE077DDE82E8D2D63E073DDC82E93
:104A7000FF248D2D6AE06EDD2A2D30E02F7030701E
:104A8000412F50E02427352764E0220F331F6A9519
:104A9000E1F792945FE095229B24922AF101919292
:104AA000282D30E02F7030702E253F2544E0220F56
:104AB000331F4A95E1F7A2943FE0A322AC24A22A37
:104AC000D1011196AC9282949FE08922882684E0DD
:104AD000EE0CFF1C8A95E1F78E288182B3E05B0E15
:104AE000852D28960FB6F894DEBF0FBECDBFCF91AF
:104AF000DF911F910F91FF90EF90DF90CF90BF90CB
:104B0000AF909F908F907F906F905F904F903F906D
:104B10002F9008952F923F924F925F926F927F92C3
:104B20008F929F92AF92BF92CF92DF92EF92FF92BD
:104B30000F931F93DF93CF9300D00F92CDB7DEB7C3
:104B40002B011C018824D101ED913D01FE2EFFE0D7
:104B5000FF22CE2EC294BFE0CB228FE06F2DFADC75
:104B6000D82E87E06C2DF6DC182F6C2D6F2589E090
:104B7000F1DCA82EA294A0EFAA221D25A12A85E08F
:104B80006F2DE8DCE82E83E06C2DE4DC182F88E044
:104B90006F2DE0DC082F8CE06C2DDCDC0827029503
:104BA000007F1E25012B8AE06C2DD4DC182F8F2D61
:104BB00067E0D0DCC8268CE06C2DCCDC982E92947B
:104BC000F0EF9F221D25912A44E050E0240E351E6F
:104BD000D3011D913D01F12EFA24BFE0FB2287E0B5
:104BE0006F2DB8DC12951F701827A294EFE0AE224B
:104BF0001A25812F67E0AEDCE82E8F2D69E0AADC54
:104C0000D82E812F69E0A6DCA82E8F2D63E0A2DCD0
:104C1000902F907FA826A29470EFA722A9260F704C
:104C2000DE240D25A02A8F2D6CE094DCE82E812F48
:104C300063E090DCC82E812F6CE08CDCD82E8F2DA9
:104C40006AE088DC992D907F082F0D250295007F62
:104C50000927EFE09E22CE249C240929812F6AE0B7
:104C600079DC9D2C929460EF9622E8269E286214AF
:104C7000730409F0ADCF5FE0D52EDA208D2D67E00B
:104C800069DCB82E8D2D69E065DC182F8D2D6CE068
:104C900061DCE82E8D2D63E05DDCC82EFF248D2DB8
:104CA0006AE058DC202F30E02F703070412F50E048
:104CB0002427352744E0220F331F4A95E1F7A294B9
:104CC0003FE0A322AB24A22AD201AC92292D30E0EE
:104CD0002F7030702E253F2594E0220F331F9A95B8
:104CE000E1F702950F700C25022B11960C9311978A
:104CF00092941FE091229826F4E0EE0CFF1CFA95A6
:104D0000E1F79E2812969C928394B5E08B1631F0C1
:104D1000E3E0F0E04E0E5F1E130115CF0F900F90F1
:104D20000F90CF91DF911F910F91FF90EF90DF9047
:104D3000CF90BF90AF909F908F907F906F905F903B
:104D40004F903F902F9008953F924F925F926F92B5
:104D50007F928F929F92AF92BF92CF92DF92EF920B
:104D6000FF920F931F93CF93DF936C013B01542E5F
:104D7000E901402EEE243324339449010894811C28
:104D8000911C22E0A22EB12CAC0EBD1EE41410F03A
:104D9000FF2410C0F6011081552021F49FE0F92E68
:104DA000F12207C0F12EF2948FE0F8220894C11C82
:104DB000D11C53240881802F8F7062E0CBDB182F29
:104DC000802F82958F7064E0C5DB8F258295807F70
:104DD0001F25812B8883F4010081802F8F7068E06C
:104DE000B9DB182F802F82958F7063E0B3DB8F259E
:104DF0008295807F1F25812BF4018083F50110812E
:104E0000812F8F7066E0A6DB082F812F82958F702F
:104E10006CE0A0DB8F258295807FF026F82AF501D3
:104E2000F082E394F9E0EF1609F0B0CFDD24EE2430
:104E3000CC24C394F3011081DD2021F40FE0F02E87
:104E4000F12207C0F12EF2941FE0F1220894611CB8
:104E5000711C0881802F8F7062E07CDB182F802FFF
:104E600082958F7064E076DB8F258295807F1F2589
:104E7000812B8883F4010081802F8F7068E06ADBCA
:104E8000182F802F82958F7063E064DB8F258295C9
:104E9000807F1F25812BF4018083F5011081812FF4
:104EA0008F7066E057DB082F812F82958F706CE042
:104EB00051DB9F2D98279295907FF0269F29F50131
:104EC0009083E394F6E0EF1611F0DC24B3CF8981F0
:104ED000982B8881892BDF91CF911F910F91FF90A3
:104EE000EF90DF90CF90BF90AF909F908F907F908A
:104EF0006F905F904F903F9008952F923F924F9206
:104F00005F926F927F928F929F92AF92BF92CF9259
:104F1000DF92EF92FF920F931F93CF93DF93EC01F9
:104F20002B01E880CE2CC294BFE0CB2219818C2DBE
:104F300090E02E2D30E02F703070822B932B212F9C
:104F400030E02F703070822B932B892B11F480E08E
:104F5000DDC0AFE08A2E8122DA80FFE06F2E6D2067
:104F6000882D662DF7DAA82E912E9294EFE09E22DE
:104F7000892D2DDBA8268C2D692DECDA382E882D75
:104F800026DB282E38268C2D662DE4DAF82E882D87
:104F9000692DE0DA082F7FE0B72EBE208B2D6A2D19
:104FA000D9DA182F882D632DD5DA782E802F8F250A
:104FB0006C2DD0DA7126782609F475C08C2D6A2DF7
:104FC000C9DAE82E8C2D03DB0D2D02950F70602FB2
:104FD000C1DA182F8B2D692D462DC6DAF82E8B2DB0
:104FE000682D402FC1DA082F822D692DB3DA1E25D6
:104FF0001F2510278127672DD6DAF20181936F01D3
:1050000009816FE0962E9022892D6A2DA3DA882ED1
:10501000F880AF2CA2945FE0A52202950F70BA80B1
:105020004FE0E42EEB208A2D602F4E2D9DDA182FB5
:10503000FFE0FF226B2C62943FE063228F2D602FF4
:10504000462D92DAB82E8E2DC2DA6F2D83DA082F14
:105050008A2D692D462D88DA18251B2510278127D2
:10506000672DA1DAF20181831A81812F82958F70D9
:10507000632D70DAF82E812F8F70A9DA682F88815E
:1050800082958F7067DA082F198112951F70812F12
:105090009EDA612F5FDA0F258027672D84DAF6010B
:1050A000818383E033C0AA2019F1862D90DA182F6E
:1050B0008D2D82958F70692D4DDA81276A2D73DAD7
:1050C000F2018083F9801A81612F62956F708F2DB4
:1050D0008F7040DA082F1F708F2D82958F70612F8F
:1050E00039DA80276A2D5FDAF201818382E00EC00F
:1050F0008C2D6B2D58DA182F882D6C2D54DAF20177
:105100008083181711F08FEF01C081E0DF91CF91FC
:105110001F910F91FF90EF90DF90CF90BF90AF90D5
:105120009F908F907F906F905F904F903F902F90C7
:105130000895BF92CF92DF92EF92FF920F931F9349
:10514000CF93DF93EC016A01623039F1633009F0EB
:1051500040C0BB24EE248E2D1FDAF82E38DA182F2B
:105160006F2DF8D9082F812F6881F4D9182F8F2D32
:105170006981F0D9102718278A81181721F4F601C0
:10518000F1926F01B394F2E0FB1520F0E3948FE00D
:10519000E81609F78B2D835020C0EE24FF248F2DB5
:1051A000FBD9082F14DA182F802F6981D3D918273B
:1051B0008881181739F4F60101936F01E394F1E047
:1051C000FE1520F0F3948FE0F81649F78E2D8250EB
:1051D00004C08881FA01808380E0DF91CF911F9124
:1051E0000F91FF90EF90DF90CF90BF9008954F9276
:1051F0005F926F927F928F929F92AF92BF92CF9267
:10520000DF92EF92FF920F931F93CF93DF933C01B6
:10521000EB012901423009F4B8C0FC01A080433001
:1052200009F0E6C0FA80E9806E2D6F258F2D92D9A6
:10523000982E6E2D8FD9082F1881812FC8D9682FED
:10524000802F88D9612F86D9D82E6E2D61278E2D7B
:1052500081D9612F7FD9082F8F2DB9D9C82E802FE2
:105260006C2D78D96F2D76D9B82E6F2D6127812FAF
:1052700071D96F2D6FD9182F8E2DA9D9082F812F95
:10528000602F68D96E2D66D9BD24B8261FE0D12EB7
:10529000DA208F2D6D2D5ED91A2D12951F70612F7A
:1052A00068278F2D57D9A82E802F6E2D53D9682FA0
:1052B0008A2D50D9082F8E2D6D2D4CD918278E2D63
:1052C000612F48D9882E8C2D6F2D44D9682F882DB9
:1052D00041D9182FF30161816F70892D4E2D44D96A
:1052E000102781276B2D5FD9F20181936F0108810F
:1052F000802F6DD9602F2ED9682F8A2D2BD9E82EBB
:10530000F3011081612F6F70802F24D912951F70C7
:105310001827802F612F1ED9982E1A81812F57D9D7
:10532000612F18D9692D16D9F82EF30181818F705C
:10533000602F10D9A82E0127812F602F0BD9682F3D
:105340008A2D08D9FE248F256B2D2DD9F20181835A
:10535000F8808F2D3CD96F2DFDD8682DFBD8E82E15
:105360001981812F34D9612FF5D8692DF3D8082FF1
:10537000F126812F6F2DEED8682F8A2DEBD80E25C0
:1053800080276B2D10D9F60131C01881812F1FD9CC
:10539000D82EF9808F2D1BD9082F8D2D6F2DDAD89F
:1053A000E82E802F612FD6D8E826F3011081812FB7
:1053B0008F70602FCFD8082F812F82958F706F2D1F
:1053C000C9D880276E2DEFD8F2018083F3011081B8
:1053D000812F8F706D2DBED8082F812F82958F70F1
:1053E0006881B8D880276E2DDED8F201818306C08F
:1053F0008A2D8F706881D7D8F2018083DF91CF9199
:105400001F910F91FF90EF90DF90CF90BF90AF90E2
:105410009F908F907F906F905F904F9008955F92D4
:105420006F927F928F929F92AF92BF92CF92DF92B4
:10543000EF92FF920F931F93DF93CF93CDB7DEB719
:105440002C970FB6F894DEBF0FBECDBF5C01842E43
:10545000022FDE011196E6E0F1E083E001900D926B
:105460008150E1F7C501482D7E010894E11CF11C33
:1054700097016ADC882319F400E010E064C024E09E
:10548000C22ED12CCC0EDD1EC701B60136DD982E02
:105490008FEF981619F40FEF10E055C08E01065FDC
:1054A0001F4FC601692DA80144DE882319F00EEFB5
:1054B00010E049C097E0692E712C6C0E7D1EC7016B
:1054C000B801492D930193DE6801730100E010E0FB
:1054D0008EE0582E34C0F601808157D8F52DF81B88
:1054E0008F2F880D8A30A8F4282F2695F7019081F8
:1054F00080FF09C0F501E20FF11D9295907F808138
:105500009827908306C0F501E20FF11D808189275D
:105510008083F701408198E020E030E0892F8423E8
:1055200011F00F5F1F4F96952F5F3F4F24303105CD
:10553000A9F70894E11CF11C0894C11CD11C8E2D04
:105540008619891540F2C8012C960FB6F894DEBF73
:105550000FBECDBFCF91DF911F910F91FF90EF90C4
:10556000DF90CF90BF90AF909F908F907F906F9083
:105570005F900895CF92DF92FF920F931F93CF9386
:10558000DF936B018C01FF24C0E0D0E0B6016C0F0B
:105590007D1FC80140E028E042DF843040F4F80E6F
:1055A0000C5F1F4F2396CF30D10581F78F2DDF91F0
:1055B000CF911F910F91FF90DF90CF900895AF9200
:1055C000BF92CF92DF92EF92FF920F931F93CF93F0
:1055D000DF935C01EB01142FFF24DD24EE2400E0B7
:1055E000CC24C39426C08F2D90E06D2D70E0153033
:1055F00050F06C0F7D1F8A0D9B1D402F29E00FDF9F
:105600001450101B0AC06C0F7D1F110F101B8A0D48
:105610009B1D402F212F03DF10E0843018F03EEF58
:10562000E32E09C0F00E94E0F90E0C2593E0D90E9C
:10563000E80E1123C1F68E2DDF91CF911F910F91AE
:10564000FF90EF90DF90CF90BF90AF900895CF93F1
:10565000DF93EC01A0E040E050E0FA01E650F24FA9
:105660007491FE01E40FF51F8081782761E020E04E
:1056700030E0862F872309F0AF5F660F2F5F3F4F23
:1056800028303105B1F74F5F5F4F4430510529F79E
:10569000A83008F4A0E08A2FDF91CF9108958627E3
:1056A000282F22952827022E269526952025022E82
:1056B000269520252770082E892F26950794279553
:1056C000902D822706942795902582270895FB0127
:1056D000DC018D9181341CF08B350CF4805E65917A
:1056E00061341CF06B350CF4605E861B611189F32C
:1056F000990B0895FB01DC010D900020E9F711974B
:1057000005900D920020E1F70895FB01DC01059062
:105710000D920020E1F70895FB01DC01415050405B
:1057200048F005900D920020C9F701C01D9241502C
:105730005040E0F70895FB01DC0102C001900D929A
:1057400041505040D8F70895DC0101C06D9341509D
:105750005040E0F70895FB01DC018D9181341CF08D
:105760008B350CF4805E619161341CF06B350CF468
:10577000605E861B611189F3990B0895FB01DC01C2
:1057800001900D920020E1F70895FB01DC014150EA
:10579000504088F08D9181341CF08B350CF4805E84
:1057A000619161341CF06B350CF4605E861B6111F5
:1057B00071F3990B0895881BFCCFFB01DC0141506C
:1057C000504048F001900D920020C9F701C01D9291
:1057D00041505040E0F70895A0E0B0E0E1EFFBE277
:1057E000B9C07C01EB018A01690109C0CE01219693
:1057F000F6010995F70181937F01015010400115D1
:105800001105A1F7CDB7DEB7E8E0C0C0A0E0B0E079
:10581000EBE0FCE29FC0EC017B018A01690109C059
:10582000CE012196F70161917F01F60109950150A2
:10583000104001151105A1F7CDB7DEB7E8E0A6C00D
:10584000FB019F01E8944230BCF04532ACF44A3091
:1058500029F497FB1EF4909581959F4F642F77272D
:105860001ED0805D8A330CF0895D8193CB01009757
:10587000A9F716F45DE251931082C90100C0DC0162
:10588000FC01672F71917723E1F7329704C07C9177
:105890006D9370836291AE17BF07C8F30895AA1B7A
:1058A000BB1B51E107C0AA1FBB1FA617B70710F00B
:1058B000A61BB70B881F991F5A95A9F7809590953D
:1058C000BC01CD01089597FB092E07260AD077FD6C
:1058D00004D0E5DF06D000201AF4709561957F4F63
:1058E0000895F6F7909581959F4F0895A1E21A2E9D
:1058F000AA1BBB1BFD010DC0AA1FBB1FEE1FFF1F74
:10590000A217B307E407F50720F0A21BB30BE40BC3
:10591000F50B661F771F881F991F1A9469F760950A
:105920007095809590959B01AC01BD01CF010895C4
:105930009111089581568A5108F48052855808952E
:105940002F923F924F925F926F927F928F929F928F
:10595000AF92BF92CF92DF92EF92FF920F931F937D
:10596000CF93DF93CDB7DEB7CA1BDB0B0FB6F8942E
:10597000DEBF0FBECDBF09942A88398848885F846E
:105980006E847D848C849B84AA84B984C884DF80DF
:10599000EE80FD800C811B81AA81B981CE0FD11DC3
:1059A0000FB6F894DEBF0FBECDBFED010895F89499
:0259B000FFCF27
:0A59B20078783A78780000000000D1
:00000001FF
